:030000000219FDE5
:03000B000200A848
:03002B000201854A
:03005B000203306D
:0300730002031D68
:1000800002030406080C10182030406080040608A3
:100090000C10182030406080A0C00003070F1F051F
:1000A000050D050305030302C2AF306308C2638573
:1000B000798AD2AF32C0D0C0E0206221E525601637
:1000C000E473E525F4C3334009758A00D263F579FA
:1000D00001D4F58AD262D0E0D0D0D2AF32C3E526C7
:1000E000334009758A00D263F57901EEF58AC26260
:1000F000E526F4602F30682520720DD0E0D0D0C204
:1001000092C296C294D2AF32C292C296C294206F6B
:100110000C206509740ED5E0FDE57B4290D0E0D05F
:10012000D0D2AF32758A00D263757900C28DD262A7
:10013000211D01C2306805206502D29201C23068DB
:1001400005206502D29401C2306805206502D2966E
:1001500001C2C29330680A2065077410D5E0FDD251
:100160009201C2C29530680A2065077410D5E0FD7F
:10017000D29401C2C29730680A2065077410D5E096
:10018000FDD29601C2C2AFC2AD53E6EFC0D0C0E00F
:10019000D2D3D2AFE57A6009E57760057577004183
:1001A000CA757701C2CEE52A6007207449152A2155
:1001B000F67800790020742EE580307E01F430E579
:1001C0000278FF53DACF207E0343DA20307E0343E8
:1001D000DA10C2D8C271E580307E01F430E50279D0
:1001E000FFC3E89970CB306103752A18207403753A
:1001F0002A18885CD27020740DE52B6004152B4101
:100200000643DA01C2D82070024179A85C2061025D
:10021000C270207431C3E894F0400374F0F8E8C46D
:10022000540F28F87984B703024146C313C31387D8
:1002300021200802C313200A06C3C898F8414628A3
:10024000F8500374FFF8C3E895655003E565F88836
:1002500022E52D54066022206B1FE536C333C333DD
:10026000F8E564C313C313F9C3952240028922E859
:100270002522F52250037522FF852224A824C3E5F8
:100280002495614002A8618825E566700241BDC3DE
:10029000E8AA669A5003E8FAE4F9EAC333FBE56892
:1002A000F45B29400D2567F8E56760021567400B90
:1002B00041BD0AC3E5679A5002056778FF8826C2E8
:1002C0006FC3E52694F84002D26F20CF0AD0E0D069
:1002D000D043E610D2AD32C2CF053AE57A6009E5E7
:1002E00078600575780061137578017801E52A60FA
:1002F00005307402152AC3E55C94014005755F0062
:100300006113756000756900E55F2401F55F5003B6
:10031000755FFFD0E0D0D043E610D2AD32C2AF530C
:10032000E67F7592FA7593FFC260759104D2AF3281
:10033000C2AF53E6EFC2ADC0D0C0E0C0F0D2D3D25E
:10034000AFA8FBA9FCE57A6007C3E913F9E813F845
:10035000C2D830710261A253DACF207E0343DA1093
:10036000307E0343DA20D271E580307E01F420E54F
:1003700002617988278928A1CF53DACF207E0343F1
:10038000DA20307E0343DA10C2D8C271307402A181
:10039000BB7800E580307E01F430E502A1BB885CCB
:1003A000A1A353DACF207E0343DA20307E0343DA61
:1003B00010C271206102817B53DACF207E0343DAC1
:1003C00010307E0343DA20C2D8D27188578958C3CF
:1003D000E89555F8E99556F97B007E087A00C3E860
:1003E000948CE994005005755B00816D882178A29A
:1003F000E6A8216055C3E894C8E994005008E4D207
:10040000E4FB7A0A8148C3E89468E994015008E45F
:10041000D2E3FB7A0F8148C3E894D0E994025008F4
:10042000E4D2E2FB7A1E8148C3E894A0E994055027
:1004300008E4D2E1FB7A3C8148C3E89498E9940847
:100440005008E4D2E0FB7A787E00C3E89559FCE9D5
:10045000955AFD30E70AECF42401FCEDF43400FD7C
:10046000755B00C3EC9AED9E5003755B018859895A
:0F0470005A8557558558567802A1A3C3E895279A
:10047F00F8E99528F9307C02A187307B02A18730FB
:10048F007A02A180207502819EE9FDE8FC81BDE919
:10049F00C313F9E813F8307902A180E9C313F9E81F
:1004AF0013F8307802A180E9C313FDE813FC206133
:1004BF002CC3EC941CED9402400281D4ED701EC34A
:1004CF00EC94C850180529E52970021529C3E529B0
:1004DF00940A5002A1BB755C00D270A1BBE52960E4
:1004EF000215297888E6F97400207F087896B903F9
:1004FF0002789EE624FAFEE43400FFC3EC9EFCED86
:10050F009FFD9208B90310A2085007207609D276F2
:10051F00A126307602C276A2085016B9030DECF46C
:10052F002401FCEDF43400FD02054078007900A1B0
:10053F0087B90315EC33FCED33FDC3EC940AFCEDE6
:10054F009400FD50047C007D00C3EC94FFED9400FB
:10055F00400678FF7900A187EC8572F0A4C5F0A260
:10056F00F733F8790040030205A378FF79000205FD
:10057F00A3E9C313F9E813F8307C0EE9600278FFA2
:10058F00C3E81338F8E43400F9C3E894FFE99400A2
:10059F00400278FF885CD270206102A1BB741FF407
:1005AF00552F4BF52FC274EB7002D274752A183089
:1005BF007403752A0A306102A1CF20740353DAFE47
:1005CF00207403752B06D0F0D0E0D0D0D2AD43E627
:1005DF00103279010205FF79030205FF790A02053E
:1005EF00FF791E0205FF79640205FF79C80205FF36
:1005FF007817E4D5E0FDD8FAD9F6227A147B780281
:10060F0006267A107B8C0206267A0D7BB40206260C
:10061F007A0B7BC8020626E573D5E001227902E446
:10062F00C295D5E0FDD294D5E0FDC294D5E0FDD2C0
:10063F0095D5E0FDE920E002D29230E002D296E5B6
:10064F0073D5E0FDE920E002C29230E002C2967459
:10065F0096D5E0FDD9C9EAF8D5E0FDD8FBDBB8C2E5
:10066F009522C37C007D0075F00005F0EA33FAEBAC
:10067F0033FB50F6EB13FBEA13FAC3E9FFE8FEE88E
:10068F009AF8E99BF95004EFF9EEF8B3EC33FCED6F
:10069F0033FDD5F0DFEDF9ECF822E889F08A20D2AE
:1006AF00D4F8A9F07B0030F70B7BFFF42401F8E9B5
:1006BF00F43400F9E88520F0A4ADF0F8E98520F0D6
:1006CF00A4AFF0FEED2EF974003FFA7C04C3EA13D9
:1006DF00FAE913F9E813F8DCF48BF030F70AE8F4D1
:1006EF002401F8E9F43400F9E889F0C2D4F8A9F04C
:1006FF002222C3E54113F9E54013F8C3E54498F806
:10070F00E54599F9500CC3E89480E994FF4016022F
:10071F000738C3E8947FE994005003020738787FC5
:10072F007900020738788079FF8849894A22E5499C
:10073F002546F8E54A3547F9854A20E4300701F4A4
:10074F003548FA30E709C3EA94F04015020776C33B
:10075F00EA940F500302077678FF79FF7A0F0207AA
:10076F0076780079007AF0C3E5249561500AC37456
:10077F00019524500B020794E54A20E70E020794D7
:10078F00E54A30E706884689478A482278A5E6FA7F
:10079F00C3E54933F8E54A33F9D1A9E930E70BC38B
:1007AF00E89480E994FF4013E1CEC3E8947FE99485
:1007BF00005002E1CE787F7900E1CE788079FFE8B2
:1007CF0020E715C3E52398F84009C3E894014003D7
:1007DF000207F578010207F5E8F424012523F84014
:1007EF00030207F578FF884B2278A6E6FAA847A9F7
:1007FF00481206A9E930E70CC3E89401E994FF40D9
:10080F001602082AC3E894FFE99400500302082A4D
:10081F0078FF790002082A780179FFE920E715C3EC
:10082F00E54B98F84009C3E894014003020851785A
:10083F0001020851E8F42401254BF8400302085146
:10084F0078FF88242278FF20692879A1E76023E5C3
:10085F0041601F74FF8541F0848539F0306A03755C
:0E086F00F005A4F8C5F0600278FFC3E89564B8
:10087D005002A864886322C3E54094C8E541940002
:10088D00E5635003140195046002F5632202089D8F
:10089D002275E890227883E6FF30EDF9A8BDA9BE58
:1008AD000570C3E57094084052757000E9FA79A09F
:1008BD00E76044EA7007E571601B0208D6C3E8954E
:1008CD00716010E5715006600C140208E20460F9C5
:1008DD000208E2E571F571C39472401B7561C0C3E6
:1008ED0094044013756180C39404400B756140C33B
:1008FD009404400375610075BB0822E561F4600244
:10090D000561E570B4070375BB1022743279A787B2
:10091D00F0A4C5F0A2F733F8C3E895614002A861D1
:10092D008822882488258826886422754000754190
:10093D00F022C2AF75C820A8CCA9CDAA3A30CF01FC
:10094D000A75C824D2AFC3EA13FAE913F9E813F80C
:10095D00AB3BAC3C883B893CC3E89BF8E99C2069E8
:10096D000A547FF9306602415C21B6AD3D8A3DF9EE
:10097D00EA9D547FFA600478FF79FFAE3EAF3F8B5E
:10098D003E8C3FA83BA93CC3E89EF8E99FF9C3E51F
:10099D004113FBE54013FAE82AF540E93BF54150D8
:1009AD00067540FF7541FF4103AA40AB41AC40AD18
:1009BD00417E047F02C3EB9404400D1E1FC3EB94D4
:1009CD00084005206A021E1FC3ED13FDEC13FCDE6B
:1009DD00F7C3EA9CFAEB9DFBEF6009C3E913F9E855
:1009ED0013F8DFF7EA28FAEB39FB8A408B41500602
:1009FD007BFF8B408B41C3EB94025002D266306972
:100A0D00047F03412E7892E6FFC3E53794824011AF
:100A1D000FC3E53794A040010FC3EF940640027F4A
:100A2D00057E02E541C4540FF9E541C454F0F8E5E3
:100A3D0040C4540F28F8C3E89EFAE99400FB40091E
:100A4D00C3EA9402EB940050047A02E4FB41A8AA95
:100A5D0040AB41EBC4FEEAC4540F4EFCC3EA9CFA12
:100A6D00EB9400FBC3E813C313F8EA28FAEB340048
:100A7D00FB8A408B41C3EB94024002C2667802EBC5
:100A8D00C4FE7B00EAC4540F4EFAC3EA98FA40053F
:100A9D00C3940250027A027892E6FF30600241A8B8
:100AAD00855192855293D26043E680C3E49AF8E46F
:100ABD009BF9C3E833F8E933F9306602613BE8FA94
:100ACD00E9FBD3E913FDE813FC88518952C3EF9478
:100ADD00036038EF20E00DE82CF8E93DF9ECFAED74
:100AED00FB020B04E828F8E939F9C3E82402F8E918
:100AFD003400F97AFE7BFFC3EF9403400E8A538BCB
:100B0D0054884D894E8C4F8D50616F885389548A0E
:100B1D004D8B4E8C4F8D503069127553F07554FFBF
:100B2D00754FF07550FF7551F07552FF616FE8FA12
:100B3D00D3E813FC8851C3EF94036020EF20E00746
:100B4D00E82CF8ECFA615BE8282402F87AFEC3EF92
:100B5D00940340088A53884D8C4F616F88538A4D9A
:100B6D008C4FE568C3335002646BF56830600261E9
:100B7D0079753402D26043E680E52D5406602DA8C8
:100B8D0040A941C3E913F9E813F8306904E9244099
:100B9D00F9C2AF53E67F759100C3E498F594E499DB
:100BAD00F595759104D26043E680D2AF22D264757B
:100BBD004300752000306C03752040020BD9D264C0
:100BCD00754300752040306C037520007801790164
:100BDD00206620E52D54066002C2647914E541C3F8
:100BED0013700104F8C3941440027814306904782A
:100BFD001B791BC3E833F8C3E933F9206010E543D3
:100C0D00600C306903D53404D26D81907181054338
:100C1D00E59BF45440B52002817A30690908C3E898
:100C2D0099400118810820640A08C3E899400261BF
:100C3D00D98108C264C2AF53E67F75910030661248
:100C4D007594007595F0759104D26043E680D2AF2E
:100C5D0061D9E5417EFFC3334009C3334005C3333A
:0E0C6D004001FEC3E49E759400F5958153C3CB
:100C7B00E5339401500261D930640261D9D8028105
:100C8B008E8108C26DC2AF53E67F75910085539478
:100C9B00855495759104854D92854E93D26043E6AC
:100CAB0080D2AFE52D54066008206A020533020C92
:100CBB00CC306D0D206C0A2064071581158102154F
:100CCB00B02278003064027801E53775F007A4F99B
:100CDB00E5F028F5F0E9A2F013A2F113A2F213F557
:100CEB0037C394785003753778C3E5379538400888
:100CFB00D265C292C296C294306002A103854F9214
:100D0B00855093D26043E68022207D16C2AF754298
:100D1B0002C295D293306202D296D2AF759F400237
:100D2B000F03C2AF754202C295D297306202D292C4
:100D3B00D2AF759F40020F03307243207D20C2AFAC
:100D4B00754203900163757B20C296C29730620493
:100D5B00D294A161D295D2AF759F41020F03C2AF5E
:100D6B00754203900163757B20C292C2933062047B
:100D7B00D294A181D295D2AF759F43020F03207DF0
:100D8B0017C2AF75420390013EC296306202D294F5
:100D9B00D2AF759F41020F03C2AF75420390013E64
:100DAB00C292306202D294D2AF759F43020F0320DE
:100DBB007D16C2AF754204C293D297306202D294B1
:100DCB00D2AF759F43020F03C2AF754204C297D2D5
:100DDB0093306202D294D2AF759F41020F033072EF
:100DEB0043207D20C2AF754205900152757B08C22E
:100DFB0094C295306204D292C107D293D2AF759F41
:100E0B0040020F03C2AF754205900174757B80C21F
:100E1B0094C295306204D296C127D297D2AF759FF8
:100E2B0040020F03207D17C2AF754205900134C2FB
:100E3B0094306202D292D2AF759F40020F03C2AFC1
:100E4B00754205900148C2943062EBD296D2AF75D1
:100E5B009F40020F03207D16C2AF754206C297D288
:100E6B0095306202D292D2AF759F41020F03C2AF8F
:100E7B00754206C293D295306202D296D2AF759F5D
:100E8B0043020F03307243207D20C2AF75420190A5
:100E9B000174757B80C292C293306204D296C1AD4D
:100EAB00D297D2AF759F43020F03C2AF7542019029
:100EBB000152757B08C296C297306204D292C1CDA3
:100ECB00D293D2AF759F41020F03207D17C2AF752E
:100EDB004201900148C292306202D296D2AF759F06
:100EEB0043020F03C2AF754201900134C2963062C8
:100EFB0002D292D2AF759F41C26522900132757BAF
:100F0B0000C292C296C294C293C297C295C2622289
:100F1B00788076FF0876FF0876FF0876FF08760361
:100F2B0008760408760A08760308760108760178B5
:100F3B008C76010876FF0876FF0876FF0876FF08A7
:100F4B0076FF0876030876FF0876FF0876FF0876AB
:100F5B00250876D00876FA0876FA0876040876FF24
:100F6B0008760108760008767A0876FF087601087D
:100F7B007601087600087603087600227887E6FF6C
:100F8B00C272BF0302D2727888E6C394036008C2B0
:100F9B007DE630E102D27DC27E7889E630E102D275
:100FAB007EC3EF94026008758E01D273020FBF757A
:100FBB008E00C273227880E6149000809378A5F699
:100FCB007881E6149000809378A6F67886E61490E4
:100FDB00008D9378A7F67886E6F539C39402500313
:100FEB00753902789CE67538FFB402037538A0B4E6
:100FFB00030375388278A3E61490009A93F5661272
:10100B000F0622227896E6FA7897E6FB7888E6B404
:10101B000305C3EB940EFB307F047A007BFFC3EB1D
:10102B009AFCC3948250027C827572000572EC8527
:10103B0072F0A4C3E5F0947D40F222D27F110F121F
:10104B0005F01205F07A007B007C101205E6E55CDA
:10105B002AFA74003BFBDCF37C04C3EB13FBEA13AF
:0F106B00FADCF7FEC27F110F22757C00757D0045
:10107A00E5EF20E6037520000520903FFFE52014E8
:10108A006006901FFF1460009304600375EF165307
:10109A00D9BF7581C043FF801205E175EF0643B2DF
:1010AA0003E5B3240220E70DF521E5E320E00685F8
:1010BA0021B343E301120F067580FF75A40075F191
:1010CA003075D4DF75900375A5FC75F2FC75D501F2
:1010DA0075A60175E241C292C296C2941205F5D272
:1010EA0093D297D2951205E1C293C297C295120F75
:1010FA0006E4F8F6D8FD756801120F1B12160A7875
:10110A00988673753001C2AF1205FA12060A1205E3
:10111A00F01206111205F01206181205F01217271E
:10112A001205FA1205FA1205F5C2AF757C00757D33
:10113A000078FA79FA308507D9FBD8F7021C001231
:10114A000F87120FC0110E110F78988673120F06AF
:10115A0075A90075B680757A00758810758902754B
:10116A00C82475910475D84075A82275B80275E629
:10117A0090759B80759D0075D10E75BCC075BB08B6
:10118A0075BA1175E8801205E1D2AF12089A753660
:10119A000053DACF207E0343DA20307E0343DA108D
:1011AA0043DA01C2D8C2711205FAD2617B037A0C02
:1011BA00E55B70077A0CDB030211331205F020702D
:1011CA0003021133C270E55CC3940240E1E52F5477
:1011DA001F855E5DF55EB55DD5DAD5C26153DACF9E
:1011EA00207E0343DA20307E0343DA10C2D8C2716C
:1011FA0078A2E67008D274E52F54E0F52FC275750F
:10120A0029001205F5307409C3E529940A4002D26F
:10121A00751205E678023074027800C3E55C9840DE
:10122A00F0C2AF12060A12060A12060AD2AF120555
:10123A00FA754C007888E6B4030261331205E67841
:10124A008CE6C394015003021333E530C394015072
:10125A0003021333757CA5757DF1207435C3E55CF3
:10126A0094FF5003021333C2AF12061FD2AF120506
:10127A00F5C3E55C940150EFC2AF12060A1205EB02
:10128A0012060AD2AF1205F5C3E55C94FF40E902E3
:10129A0017AC7F05D27F110F1205F5C2AFC27F11BD
:1012AA000FAE5CC3E55C947FD2AF50026143120576
:1012BA00E1C2AF12061FD2AFDFDA1146C3EE9405C0
:1012CA007897F61205FA12172F7F0AD27F110F129A
:1012DA0005F5C2AFC27F110FAE5CC3E55C947FD245
:1012EA00AF50E61205E1C2AF12060A1205EB12066A
:1012FA000AD2AFDFD61146EE24037896F6F879972C
:10130A00E7C394824003985006E824827897F6123D
:10131A0005FA12164C12175E1205F5110FC3E55C99
:10132A0094FF5002415E0217AC757C00757D00C3C4
:10133A00E55C954C4003855C4C1205F5780179888B
:10134A00E7B403027805C3E55C984002413EC2AFA8
:10135A0012061F12061F12061FD2AF1205FA7530A7
:10136A0000E4F531F5320531E531F4703F053278A4
:10137A009AE67819146012783214600D787D146038
:10138A000878FA146003753200C3E53298401D12DA
:10139A000F061205E1153275310078998673C2AFCE
:1013AA0012061FD2AF789886731205F51205EBE57F
:1013BA002A7005307402213378012074027806C33A
:1013CA00E55C9840A17888E6C3940360031205F5AA
:1013DA00E52A7003021133C2AF120F06E4F522F5B3
:1013EA0023F524F525F526F567D2AF7885E6C333CC
:1013FA00F565E4F544F545F546F547F548F570F524
:10140A002CF52DF53775700875BB101205E1120819
:10141A009E30EDFDA8BDA9BEE97001F888711208D9
:10142A00A275700875BB10120F87C2AF7561FF12E3
:10143A000918852261852262852263D2AF7522014D
:10144A00752401752501752601856069756A01751E
:10145A00B69075A903757A017888E6B40307C27D48
:0F146A00307602D27DD268D269753300120E60DF
:10147900120E8F12093812093F12093812093F1248
:101489000938120BCB120700120CCD120D141209D8
:101499003F120BBA306E031207012066031208547B
:1014A900306603120884120CCD120D4312093F1243
:1014B9000BCB306E0312073D120CCD120DBA120977
:1014C9003F120BBA306E0312079B120CCD120DE9B5
:1014D90012093F120BCB306E031207F8120CCD1212
:1014E9000E6012093F12089E120BBA120CCD120E91
:1014F9008F1208A212093F30692F856461856462E1
:10150900856069756A0179187A0CC3E53399400CCD
:10151900C269D26A8A357561FF021532C3E55C94E6
:1015290001400302148B0215B8306A1D206C1AE5BC
:1015390035147006C26AD26B818BF535C3E55C94AC
:1015490001400302148B0215B8753600788279A41C
:10155900E760027803C3E55F985054307404E52AC4
:10156900604D7888E6B40317207D05207607A188A9
:10157900307602A188206C07D26C85646181CA78B3
:10158900F0306C058564617820C3E541985002818B
:101599008B306C1BC26CC27D307602D27DD26A75EB
:1015A9003512856461818B0536E55C6002A1BB75E6
:1015B9003600C2AF120F067887E6FE7602120F8751
:1015C9007887EEF6E4F522F523F524F525F526F5D9
:1015D90065752C00752D0075A90075B680757A00A2
:1015E900D2AF1205F5120F0678A4E66006D293D29F
:1015F90095D297307409C3E53694044002213361CA
:101609006B901A0D782012168EE520B45A0CA3128D
:10161900168EE520B4A50302162C120F1B12164CC8
:1016290002164B901A0378807B0A12168EA308DBE8
:10163900F9901A0F788C7B1912168EA308DBF99092
:101649001A2822C2AF1216D11216AE901A00740EC1
:10165900121693A37407121693A374151216939076
:101669001A0378807B0A121692A308DBF9901A0FE5
:10167900788C7B19121692A308DBF91216E412165C
:10168900C2901A2822E493F622E6438F01538FFD74
:10169900FFC3E583941C400122EF857CB7857DB7A4
:1016A900F0538FFE22438F02438F01857CB7857DDE
:1016B900B7901A0DF0538FFC22901A0D745AD193DA
:1016C900901A0E74A5D193227A3079D07820901A85
:1016D90040D18EE520F709A3DAF7227A3079D09044
:1016E9001A40E7D19309A3DAF922AB74A875BB01B3
:1016F900027984BB02027985BB03027986BB0402A5
:101709007992BB05027987BB060279A3BB070279E7
:101719009CBB08027988BB09027989E8F7227C0514
:101729001205FADCFB22C2AF12060A1206111206D2
:101739001812061F1205EB12060A120611120618D4
:1017490012061F1205EB12060A12061112061812CA
:10175900061FD2AF22C2AF12061F120618120611B7
:1017690012060A1205EB12061F12061812061112AA
:10177900060A1205EB12061F1206181206111206A6
:101789000AD2AF22AE74AF75C2AF12060A12060AA8
:1017990012060A1205EBDEF212061F1205EBDFF83C
:1017A900D2AF22F12FF127F12775740175750175F3
:1017B9007600F18D7C05AD5C1205FAC3ED955C7080
:1017C900F5C3E55C9401400AC3E55C94FF4032022D
:1017D90017E8D1F3D14CF12FC2AF75EF16F127DC21
:1017E900D50576C3E5769403500280C6F1270575C1
:1017F900E5741490009F93F808C3E575985002802A
:10180900AE1217271217270574C3E574940A5002FC
:10181900809A120F1B12164CC2AF75EF16121727BA
:0319FD0002107461
:101A00000E0715FFFFFFFF03040A0301015AA5019A
:101A1000FFFFFFFFFF03FFFFFF25D0FAFA04FF01DE
:091A2000007AFF0101000300FF40
:101A400023475F556C74726132304123202020207F
:101A500023424C48454C492346333930232020202B
:101A60002020202020202020202020202020202076
:101C0000C2AFC2D353D9BF7581C043B20343FF8073
:101C1000752438752503B1DC7529A5752AF175E29F
:101C20004043F12053A4DF75D4FFD2857DFA7803B9
:101C300079E67C10752200752300901DE97B0675FE
:101C400024987525013085028145208508D8FBD967
:101C5000F9DCF781B7308508D8FBD9F9DCF781B713
:101C6000B19CE493A3C39A6004DDC381B7DBDBB10D
:101C70008E6002812E7B08E493FAA3B16FDBF87AC1
:101C800030B16F752200752300B18EEAFCEBFDC305
:101C9000ED94FE400EB18E8A278B28ED30E0048A49
:101CA000828B83B18E7AC270D8C3ED94FE601950D6
:101CB000CEBD002BEC600F7520007521FF7529004B
:101CC000752A000200008100A827A9280809D80465
:101CD000D90281DCB192EA89AAF281CE0D81A3C337
:101CE000ED94035053EDA2E092007AC5C3E58294CF
:101CF00000E583941C508A200010438F02438F011B
:101D00008529B7852AB7F0300029A827A92808090E
:101D1000438F01538FFDD804D902A133C3E58394C7
:101D20001C4003A3A11689AAE28529B7852AB7F02A
:101D3000A3A116538FFC817F7AC1BD030CE493A34A
:101D4000FAB153DCF8B14B817F8181AA22AB23B178
:101D50006FEBFAEA6222752608C3E52313F523E543
:101D60002213F52250066323A0632201D526EAB18F
:101D7000DCB1DC75260AEAF4200102D285300102CA
:101D8000C285B1DCC3134002C201D526EB22B19259
:101D9000EAFB208502A192308502A197752608AE44
:101DA00024AF25C3EF13FFEE13FEB1E0B1DCC3EAAD
:101DB000133085024480FA30E703632201C3E52330
:101DC00013F523E52213F52250066323A0632201B5
:101DD000D526D9E52265236523F52222AE24AF2539
:101DE0000E0FDEFEDFFCD20122424C48656C6934E6
:071DF000373163F390060197
:00000001FF
